:020000040000FA
:08000000803102288731FD2F39
:100C76007430210099008C018D0120008C018D01BA
:100C8600E1302000A0001030A1008631F826863120
:100C9600432E80310228F401F501701C532E542E88
:100CA600582E7208F4077308F53D0130F235F30D3E
:100CB600890B592E0130F136F00C890B5E2E700827
:100CC6007104031D672E682E502E7508F1007408F6
:100CD600F0000800FB01FC01760877040319742E66
:100CE600752EA42EFD01FD0A812E0130F635F70D75
:100CF600890B792E0130FA007A08FD07F71F842E3A
:100D0600852E782E0130FB35FC0D890B862E770853
:100D16007902031D902E76087802031C932E942EDA
:100D2600992E7608F8027708F93B7B140130F736DE
:100D3600F60C890B9A2E0130FD02031DA32EA42E5C
:100D4600852E7C08F7007B08F6000800D22E483076
:100D560020008D00F72EEB3020008D00F72E8C3012
:100D660020008D00F72E893020008D00F72E2B30C5
:100D760020008D00F72E193020008D00F72E183038
:100D860020008D00F72ECB3020008D00F72E083086
:100D960020008D00F72E093020008D00F72E7108F7
:100DA600003A0319D72EF72E7008003A0319AA2E17
:100DB600013A0319AE2E033A0319B22E013A03196A
:100DC600B62E073A0319BA2E013A0319BE2E033A74
:100DD6000319C22E013A0319C62E0F3A0319CA2E59
:100DE600013A0319CE2EF72E080020002108B10083
:100DF6002008B000E830F6000330F7003108F900AB
:100E06003008F80086316D26863177082000AF005D
:100E16007608AE002108B1002008B0006430F60064
:100E26000030F7002F08F1002E08F0001830F2000D
:100E3600FC30F30086314E268631200030087007DC
:100E4600F8003108713DF90086316D268631770844
:100E56002000AD007608AC002108B1002008B000E3
:100E66000A30F6000030F7002F08F1002E08F000D7
:100E76001830F200FC30F30086314E2686317008B9
:100E86002000A2007108A3002D08F1002C08F00034
:100E96009C30F200FF30F30086314E268631700812
:100EA60020002207A4007108233DA500300824076E
:100EB600F8003108253DF90086316D268631770820
:100EC6002000AB007608AA002108B1002008B00077
:100ED6002F08F1002E08F0001830F200FC30F30065
:100EE60086314E26863170082000A2007108A300C4
:100EF6002D08F1002C08F0009C30F200FF30F300C2
:100F060086314E268631700820002207A40071081B
:100F1600233DA5002B08F1002A08F000F630F20068
:100F2600FF30F30086314E268631700820002407F4
:100F3600A6007108253DA70030082607A80031083D
:100F4600273DA900FF308C002908F1002808F00091
:100F56008631A9268631FE3020008C000330200021
:100F6600A2009730890BB52FA20BB52F0032FF30A8
:100F760020008C002B08F1002A08F0008631A926F3
:100F86008631FD3020008C0003302000A20097300F
:100F9600890BCB2FA20BCB2F0032FF3020008C0009
:100FA6002D08F1002C08F0008631A9268631FB3089
:100FB60020008C0003302000A2009730890BE12F1F
:100FC600A20BE12F0032FF3020008C002F08F10029
:100FD6002E08F0008631A9268631F73020008C00D5
:100FE60003302000A2009730890BF72FA20BF72FB2
:0A0FF60000320800200086313B2E77
:020000040001F9
:04000E00A4D9FFDC96
:00000001FF
